:030000000219FDE5
:03000B000200AA46
:03002B0002018748
:03005B000203415C
:0300730002032E57
:1000800002030406080C10182030406080040608A3
:100090000C10182030406080A0C00003070F1F0D17
:1000A0000D04050D050305030302C2AF306308C24A
:1000B0006385798AD2AF32C0D0C0E0206221E525C5
:1000C0006016E473E525F4C3334009758A00D263F2
:1000D000F57901D6F58AD262D0E0D0D0D2AF32C362
:1000E000E526334009758A00D263F57901F0F58A77
:1000F000C262E526F4602F30682520720DD0E0D072
:10010000D0C292C296C294D2AF32C292C296C29468
:10011000206F0C206509740ED5E0FDE57B4290D080
:10012000E0D0D0D2AF32758A00D263757900C28D2B
:10013000D262211F01C4306805206502D29201C439
:10014000306805206502D29401C43068052065023C
:10015000D29601C4C29330680A2065077410D5E0B6
:10016000FDD29201C4C29530680A2065077410D58B
:10017000E0FDD29401C4C29730680A20650774106C
:10018000D5E0FDD29601C4C2AFC2AD53E6EFC0D0F8
:10019000C0E0D2D3D2AFE57A6009E5776005757724
:1001A0000041DB757701C2CEE52A600720744F1548
:1001B0002A21FE7800790020742EE580307E01F43B
:1001C00030E50278FF53DACF207E0343DA20307E19
:1001D0000343DA10C2D8C271E580307E01F430E505
:1001E0000279FFC3E89970CB306103752A18207437
:1001F00003752A18885CD270E86003755F0020746C
:100200000DE52B6004152B410E43DA01C2D8207096
:1002100002417DA85C206102C2702074367982B7E9
:100220000431C3E894F0400374F0F8E8C4540F2894
:10023000F87984B703024153C313C31387212008FD
:1002400002C313200A06C3C898F8415328F8500384
:1002500074FFF88822E52D54066022206B1FE536D6
:10026000C333C333F8E564C313C313F9C395224002
:10027000028922E82522F52250037522FF7882B6F2
:100280000459852224A824C3E52495614002A8616D
:10029000C3E895634002A8638825E566700241CEF5
:1002A000C3E8AA669A5003E8FAE4F9EAC333FBE527
:1002B00068F45B29400D2567F8E567600215674023
:1002C0000B41CE0AC3E5679A5002056778FF88267E
:1002D000C26FC3E52694F84002D26F20CF0AD0E067
:1002E000D0D043E610D2AD32C2CF053AE57A6009EC
:1002F000E578600575780061247578017801E52A54
:100300006005307402152AC3E55C94014005755FF1
:10031000006124756000756900E55F2401F55F5098
:1003200003755FFFD0E0D0D043E610D2AD32C2AF4C
:1003300053E67F7592FA7593FFC260759104D2AF50
:1003400032C2AF53E6EFC2ADC0D0C0E0C0F0D2D3EE
:10035000D2AFA8FBA9FCE57A6007C3E913F9E8135B
:10036000F8C2D830710261B353DACF207E0343DA8A
:1003700010307E0343DA20D271E580307E01F42014
:10038000E502618A88278928A1E053DACF207E031D
:1003900043DA20307E0343DA10C2D8C271307402CF
:1003A000A1CC7800E580307E01F430E502A1CC8854
:1003B0005CA1B453DACF207E0343DA20307E0343BE
:1003C000DA10C271206102818C53DACF207E0343A0
:1003D000DA10307E0343DA20C2D8D27188578958A8
:1003E000C3E89555F8E99556F97B007E087A00C375
:1003F000E8948CE994005005755B00817E88217833
:10040000A2E6A8216055C3E894C8E994005008E426
:10041000D2E4FB7A0A8159C3E89468E99401500850
:10042000E4D2E3FB7A0F8159C3E894D0E9940250F7
:1004300008E4D2E2FB7A1E8159C3E894A0E994054E
:100440005008E4D2E1FB7A3C8159C3E89498E994DE
:10045000085008E4D2E0FB7A787E00C3E89559FCA6
:10046000E9955AFD30E70AECF42401FCEDF4340080
:0E047000FD755B00C3EC9AED9E5003755B01B9
:10047E008859895A8557558558567802A1B4C3E8CC
:10048E009527F8E99528F9307C02A198307B02A1D6
:10049E0098307A02A19120750281AFE9FDE8FC81C6
:1004AE00CEE9C313F9E813F8307902A191E9C31329
:1004BE00F9E813F8307802A191E9C313FDE813FCB3
:1004CE0020612CC3EC941CED9402400281E5ED708A
:1004DE001EC3EC94C850180529E52970021529C3CE
:1004EE00E529940A5002A1CC755C00D270A1CCE52E
:1004FE0029600215297888E6F97400207F0878961D
:10050E00B90302789EE624FAFEE43400FFC3EC9EA3
:10051E00FCED9FFD9208B90310A208500720760942
:10052E00D276A137307602C276A2085016B9030DE4
:10053E00ECF42401FCEDF43400FD02055178007951
:10054E0000A198B90315EC33FCED33FDC3EC940A0E
:10055E00FCED9400FD50047C007D00C3EC94FFED97
:10056E009400400678FF7900A198EC8572F0A4C53E
:10057E00F0A2F733F8790040030205B478FF790052
:10058E000205B4E9C313F9E813F8307C0EE96002F2
:10059E0078FFC3E81338F8E43400F9C3E894FFE9B0
:1005AE009400400278FF885CD270206102A1CC7466
:1005BE001FF4552F4BF52FC274EB7002D274752AAF
:1005CE0018307403752A0A306102A1E020740353B7
:1005DE00DAFE207403752B06D0F0D0E0D0D0D2AD69
:1005EE0043E6103279010206107903020610790AE9
:1005FE00020610791E020610796402061079C802EE
:10060E0006107817E4D5E0FDD8FAD9F6227A147BD5
:10061E00780206377A107B8C0206377A0D7BB4028D
:10062E0006377A0B7BC8020637E573D5E0012279CF
:10063E0002E4C295D5E0FDD294D5E0FDC294D5E09A
:10064E00FDD295D5E0FDE920E002D29230E002D253
:10065E0096E573D5E0FDE920E002C29230E002C2D9
:10066E00967496D5E0FDD9C9EAF8D5E0FDD8FBDB46
:10067E00B8C29522C37C007D0075F00005F0EA3308
:10068E00FAEB33FB50F6EB13FBEA13FAC3E9FFE880
:10069E00FEE89AF8E99BF95004EFF9EEF8B3EC3363
:1006AE00FCED33FDD5F0DFEDF9ECF822E889F08AA8
:1006BE0020D2D4F8A9F07B0030F70B7BFFF4240195
:1006CE00F8E9F43400F9E88520F0A4ADF0F8E985F6
:1006DE0020F0A4AFF0FEED2EF974003FFA7C04C3B7
:1006EE00EA13FAE913F9E813F8DCF48BF030F70AA1
:1006FE00E8F42401F8E9F43400F9E889F0C2D4F8FA
:10070E00A9F0227882B6040302076CC3E55C94015B
:10071E004003020736852224E4F544F545F546F5F7
:10072E0047F548C26E02076C7882E6FCD26EE5226F
:10073E00F523783879C7AA40AB41C3EB13FBEA1314
:10074E00FAEC146013C3EB13FBEA13FAEC14146007
:10075E0007C3EB13FBEA13FAD1828844894522C3FF
:10076E00E5449523F8E5459400F9500CC3E89480D0
:10077E00E994FF401602079DC3E8947FE994005068
:10078E000302079D787F790002079D788079FF88A4
:10079E0049894A22E5492546F8E54A3547F9854A09
:1007AE0020E4300701F43548FA30E709C3EA94F043
:1007BE0040150207DBC3EA940F50030207DB78FFF4
:1007CE0079FF7A0F0207DB780079007AF0C3E5240F
:1007DE009561500AC374019524500B0207F9E54A3E
:1007EE0020E70E0207F9E54A30E706884689478A70
:1007FE00482278A5E6FAC3E54933F8E54A33F912FB
:10080E0006BAE930E70BC3E89480E994FF40130180
:10081E0034C3E8947FE9940050020134787F790064
:10082E000134788079FFE820E715C3E52398F84076
:10083E0009C3E89401400302085B780102085BE8F3
:10084E00F424012523F8400302085B78FF884B222D
:10085E0078A6E6FAA847A9481206BAE930E70CC30B
:0F086E00E89401E994FF4016020890C3E894FF54
:10087D00E99400500302089078FF790002089078FF
:10088D000179FFE920E715C3E54B98F84009C3E866
:10089D00940140030208B778010208B7E8F4240177
:1008AD00254BF840030208B778FF88242278FF20F3
:1008BD00692879A1E76023E541601F74FF8541F048
:1008CD00848539F0306A0375F005A4F8C5F060022F
:1008DD0078FFC3E895645002A864886322C3E5409D
:1008ED0094C8E5419400E56350031401FB046002D4
:1008FD00F563220209032275E890227883E6FF3022
:10090D00EDF9A8BDA9BE0570C3E5709408405275F8
:10091D007000E9FA79A0E76044EA7007E571601BA1
:10092D0002093CC3E895716010E5715006600C1426
:10093D000209480460F9020948E571F571C3947222
:10094D00401B7561C0C394044013756180C394044A
:10095D00400B756140C39404400375610075BB087D
:10096D0022E5612410500274FFF5617982B704020B
:10097D002195C3A861E524985002A824C3E8956386
:10098D004002A86388258826E570B4070375BB105F
:10099D0022743279A787F0A4C5F0A2F733F8C3E823
:1009AD0095614002A861882288248825882688645C
:1009BD00227540007541F022C2AF75C820A8CCA9A0
:1009CD00CDAA3A30CF010A75C824D2AFC3EA13FAC3
:1009DD00E913F9E813F8AB3BAC3C883B893CC3E821
:1009ED009BF8E99C20690A547FF930660241E44185
:1009FD003EAD3D8A3DF9EA9D547FFA600678FF7958
:100A0D00FF4123AE3EAF3F8B3E8C3FA83BA93CC37D
:100A1D00E89EF8E99FF9C3E54113FBE54013FAE8B9
:100A2D002AF540E93BF54150067540FF7541FF4100
:100A3D008BAA40AB41AC40AD417E047F02C3EB9429
:100A4D0004400D1E1FC3EB94084005206A021E1FB3
:100A5D00C3ED13FDEC13FCDEF7C3EA9CFAEB9DFB33
:100A6D00EF6009C3E913F9E813F8DFF7EA28FAEBA9
:100A7D0039FB8A408B4150067BFF8B408B41C3EB8A
:100A8D0094025002D2663069047F0341B67892E633
:100A9D00FFC3E537948240110FC3E53794A04001A1
:100AAD000FC3EF940640027F057E02E541C4540F4B
:100ABD00F9E541C454F0F8E540C4540F28F8C3E8F3
:100ACD009EFAE99400FB4009C3EA9402EB940050AE
:100ADD00047A02E4FB6130AA40AB41EBC4FEEAC4E8
:100AED00540F4EFCC3EA9CFAEB9400FBC3E813C30E
:100AFD0013F8EA28FAEB3400FB8A408B41C3EB94E0
:100B0D00024002C2667802EBC4FE7B00EAC4540FB9
:100B1D004EFAC3EA98FA4005C3940250027A02785D
:100B2D0092E6FF3060026130855192855293D2601A
:100B3D0043E680C3E49AF8E49BF9C3E833F8E9335C
:100B4D00F930660261C3E8FAE9FBD3E913FDE81356
:100B5D00FC88518952C3EF94036038EF20E00DE813
:100B6D002CF8E93DF9ECFAEDFB020B8CE828F8E9DD
:100B7D0039F9C3E82402F8E93400F97AFE7BFFC3A2
:100B8D00EF9403400E8A538B54884D894E8C4F8DB4
:100B9D005061F7885389548A4D8B4E8C4F8D503050
:100BAD0069127553F07554FF754FF07550FF7551FF
:100BBD00F07552FF61F7E8FAD3E813FC8851C3EFE3
:100BCD0094036020EF20E007E82CF8ECFA61E3E8ED
:100BDD00282402F87AFEC3EF940340088A53884D07
:100BED008C4F61F788538A4D8C4FE568C3335002A3
:100BFD00646BF5683060028101753402D26043E6A2
:100C0D0080E52D5406602DA840A941C3E913F9E8EC
:100C1D0013F8306904E92440F9C2AF53E67F7591AA
:100C2D0000C3E498F594E499F595759104D2604369
:100C3D00E680D2AF22D264754300752000306C037C
:100C4D00752040020C61D264754300752040306CF4
:100C5D000375200078017901206620E52D5406608A
:0E0C6D0002C2647914E541C313700104F8C398
:100C7B00941440027814306904781B791BC3E83351
:100C8B00F8C3E933F9206010E543600C306903D5F4
:100C9B003404D26DA11891090543E59BF45440B57A
:100CAB002002A10230690908C3E89940011881901C
:100CBB0020640A08C3E899400281618190C264C232
:100CCB00AF53E67F7591003066127594007595F001
:100CDB00759104D26043E680D2AF8161E5417EFF1E
:100CEB00C3334009C3334005C3334001FEC3E49E05
:100CFB00759400F59581DBC3E53394015002816156
:100D0B003064028161D802A1168190C26DC2AF53CB
:100D1B00E67F759100855394855495759104854DA7
:100D2B0092854E93D26043E680D2AFE52D54066098
:100D3B0008206A020533020D54306D0D206C0A2019
:100D4B00640715811581021633227800306402780E
:100D5B0001E53775F007A4F9E5F028F5F0E9A2F005
:100D6B0013A2F113A2F213F537C39478500375371E
:100D7B0078C3E53795384008D265C292C296C294C3
:100D8B00306002A18B854F92855093D26043E680F1
:100D9B0022207D16C2AF754202C295D293306202F9
:100DAB00D296D2AF759F40020F8CC2AF754202C272
:100DBB0095D297306202D292D2AF759F40020F8CC0
:100DCB00307243207D20C2AF754203900165757B65
:100DDB0020C296C297306204D294A1E9D295D2AFC9
:100DEB00759F41020F8CC2AF754203900165757BF5
:100DFB0020C292C293306204D294C109D295D2AF71
:100E0B00759F43020F8C207D17C2AF754203900173
:100E1B0040C296306202D294D2AF759F41020F8CC2
:100E2B00C2AF754203900140C292306202D294D29B
:100E3B00AF759F43020F8C207D16C2AF754204C263
:100E4B0093D297306202D294D2AF759F43020F8C2C
:100E5B00C2AF754204C297D293306202D294D2AF22
:100E6B00759F41020F8C307243207D20C2AF7542BB
:100E7B0005900154757B08C294C295306204D292DE
:100E8B00C18FD293D2AF759F40020F8CC2AF754208
:100E9B0005900176757B80C294C295306204D29620
:100EAB00C1AFD297D2AF759F40020F8C207D17C276
:100EBB00AF754205900136C294306202D292D2AF26
:100ECB00759F40020F8CC2AF75420590014AC294C8
:100EDB003062EBD296D2AF759F40020F8C207D16FD
:100EEB00C2AF754206C297D295306202D292D2AF90
:100EFB00759F41020F8CC2AF754206C293D29530DB
:100F0B006202D296D2AF759F43020F8C307244208F
:100F1B007D20C2AF754201900176757B80C292C273
:100F2B0093306204D296E135D297D2AF759F4302CC
:100F3B000F8CC2AF754201900154757B08C296C2EB
:100F4B0097306205D292020F56D293D2AF759F4162
:100F5B00020F8C207D17C2AF75420190014AC292DD
:100F6B00306202D296D2AF759F43020F8CC2AF751F
:100F7B004201900136C296306202D292D2AF759F77
:100F8B0041C26522900134757B00C292C296C29415
:100F9B00C293C297C295C2622278807609087609FD
:100FAB000876040876FF0876030876FF08760A08A9
:100FBB007603087601087601788C76010876FF08AF
:100FCB0076FF0876FF0876FF0876FF08760308762B
:100FDB00FF0876FF0876FF0876250876D008762876
:100FEB000876500876040876FF0876020876000823
:100FFB00767A0876FF08760108760108760008767F
:10100B0003087600227887E6FFC272BF0302D27212
:10101B007888E6C394036008C27DE630E102D27D96
:10102B00C27E7889E630E102D27EC3EF940260087B
:10103B00758E01D273021048758E00C273227880B0
:10104B00E6149000809378A5F67881E614900080E2
:10105B009378A6F67886E61490008D9378A7F678A9
:0F106B0086E6F539C394025003753902789CE686
:10107A007538FFB402037538A0B403037538827853
:10108A00A3E61490009A93F566120F8F222278969F
:10109A00E6FA7897E6FB7888E6B40305C3EB940E84
:1010AA00FB307F047A007BFFC3EB9AFCC394825027
:1010BA00027C827572000572EC8572F0A4C3E5F0B9
:1010CA00947D40F222D27F11981206011206017A0B
:1010DA00007B007C101205F7E55C2AFA74003BFBE2
:1010EA00DCF37C04C3EB13FBEA13FADCF7FEC27FE2
:1010FA00119822757C00757D00E5EF20E6037520C6
:10110A00000520903FFFE520146006901FFF146041
:10111A00009304600375EF1653D9BF7581C043FF6E
:10112A00801205F275EF0643B203E5B3240220E705
:10113A000DF521E5E320E0068521B343E301120F13
:10114A008F7580FF75A40075F13075D4DF75900333
:10115A0075A5FC75F2FC75D50175A60175E241C24B
:10116A0092C296C294120606D293D297D2951205CB
:10117A00F2C293C297C295120F8FE4F8F6D8FD75A2
:10118A006801120FA412168C78988673753001C202
:10119A00AF12060B12061B120601120622120601D4
:1011AA00120629120601C2AF757C00757D0078FA15
:1011BA0079FA308507D9FBD8F7021C0011101149BA
:1011CA001197119878988673120F8F75A90075B6C2
:1011DA0080757A0075881075890275C8247591041E
:1011EA0075D84075A82275B80275E690759B80750A
:1011FA009D0075D10E75BCC075BB0875BA1175E82E
:10120A00801205F2D2AF12090075360053DACF20E8
:10121A007E0343DA20307E0343DA1043DA01C2D870
:10122A00C27112060BD2617B037A0CE55B70077AF6
:10123A000CDB030211B01206012070030211B0C2C6
:10124A0070E55CC3940240E1E52F541F855E5DF5AD
:10125A005EB55DD5DAD5C26153DACF207E0343DAB3
:10126A0020307E0343DA10C2D8C27178A2E6700831
:10127A00D274E52F54E0F52FC275752900120606BF
:10128A00307409C3E529940A4002D2751205F77829
:10129A00023074027800C3E55C9840F0C2AF1206CF
:1012AA001B12061B12061BD2AF12060B754C0078D6
:1012BA0088E6B4030261AC1205F7788CE6C39401A0
:1012CA0050030213ACE530C3940150030213AC750A
:1012DA007CA5757DF1207435C3E55C94FF5003024B
:1012EA0013ACC2AF120630D2AF120606C3E55C9445
:1012FA000150EFC2AF12061B1205FC12061BD2AF39
:10130A00120606C3E55C94FF40E90218447F02D244
:10131A007F1198120606C2AFC27F1198AE5CC3E570
:10132A005C947FD2AF500261BC1205F2C2AF1206C2
:10133A0030D2AFDFDA11CFC3EE7897F612060B126E
:10134A0017C77F0AD27F1198120606C2AFC27F1151
:10135A0098AE5CC3E55C947FD2AF50E61205F2C248
:10136A00AF12061B1205FC12061BD2AFDFD611CF35
:10137A00EE24037896F6F87997E7C39482400398A7
:10138A005006E824827897F612060B1216DA12171C
:10139A00F61206061198C3E55C94FF500241D90281
:1013AA001844757C00757D00C3E55C954C40038547
:1013BA005C4C12060678017988E7B403027805C303
:1013CA00E55C98400241B9C2AF12063012063012EB
:1013DA000630D2AF12060B753000E4F531F532054E
:1013EA0031E531F4703F0532789AE67819146012C3
:1013FA00783214600D787D14600878FA14600375E9
:10140A003200C3E53298401D120F8F1205F21532D1
:10141A0075310078998673C2AF120630D2AF7898C8
:10142A0086731206061205FCE52A7005307402213D
:10143A00B078012074027806C3E55C9840A17888E8
:10144A00E6C394036003120606E52A70030211B08C
:10145A00C2AF120F8FE4F522F523F524F525F52600
:0E146A00F567D2AF7885E6C333F565E4F54447
:10147800F545F546F547F548F570F52CF52DF537A2
:1014880075700875BB101205F212090430EDFDA83D
:10149800BDA9BEE97001F888711209087570087550
:1014A800BB101110C2AF7561FF12099E85226185BC
:1014B8002262852263D2AF75220175240175250148
:1014C800752601856069756A0175B69075A90375F9
:1014D8007A017888E6B40307C27D307602D27DD2DD
:1014E80068D269753300120EE8120F171209BE127E
:1014F80009C51209BE1209C51209BE120C531207FA
:1015080011120D55120D9C1209C5120C42306E03B2
:1015180012076D2066031208BA3066031208EA1231
:101528000D55120DCB1209C5120C53306E0312075C
:10153800A2120D55120E421209C5120C42306E034A
:10154800120800120D55120E711209C5120C5330F3
:101558006E0312085E120D55120EE81209C5120923
:1015680004120C42120D55120F171209081209C560
:10157800306932856461856462856069756A01795C
:10158800187A0CC3E53399400FC269D26A8A358547
:1015980064618564630215ADC3E55C940140030290
:1015A800150302163B306A25206C22E535147006B7
:1015B800C26AD26BA103F535C3E55C94014003020E
:1015C80015037888E6C39403600302163B7536005A
:1015D80078FA79A4E760027803C3E55F985054303D
:1015E8007404E52A604D7888E6B40317207D052049
:1015F8007607C10B307602C10B206C07D26C85646C
:1016080061A14278F0306C058564617820C3E541BA
:10161800985002A103306C1BC26CC27D307602D296
:101628007DD26A753512856461A1030536E55C6073
:1016380002C13E753600C2AF120F8F7887E6FE767C
:101648000211107887EEF6E4F522F523F524F52546
:10165800F526F565752C00752D0075A90075B68001
:10166800757A00D2AF120606120F8F78A4E66006CC
:10167800D293D295D297307409C3E53694044002C8
:1016880021B061E4901A0D782012171CE520B4559A
:101698000CA312171CE520B4AA030216BA757CA580
:1016A800757DF1120FA41216DA757C00757D0002A3
:1016B80016D9901A0378807B0A12171CA308DBF945
:1016C800901A0F788C7B1912171CA308DBF9901A53
:1016D8002822C2AF12175F12173C901A00740E121C
:1016E8001721A37409121721A37415121721901A30
:1016F8000378807B0A121720A308DBF9901A0F7869
:101708008C7B19121720A308DBF9121772121750D5
:10171800901A2822E493F622E6438F01538FFDFFA7
:10172800C3E583941C400122EF857CB7857DB7F023
:10173800538FFE22438F02438F01857CB7857DB787
:10174800901A0DF0538FFC22901A0D7455F12190C8
:101758001A0E74AAF121227A3079D07820901A4092
:10176800F11CE520F709A3DAF7227A3079D0901A2C
:1017780040E7F12109A3DAF922AB74A875BB01028D
:101788007980BB02027981BB03027982BB040279AA
:1017980084BB05027986BB06027992BB070279876A
:1017A800BB080279A3BB0902799CBB0A027988BBF2
:1017B8000B027989E8F7227C0512060BDCFB22C2B2
:1017C800AF12061B1206221206291206301205FC59
:1017D80012061B1206221206291206301205FC12E6
:1017E800061B120622120629120630D2AF22C2AFF9
:1017F80012063012062912062212061B1205FC12C6
:10180800063012062912062212061B1205FC1206C1
:101818003012062912062212061BD2AF22AE74AF6E
:1018280075C2AF12061B12061B12061B1205FCDE40
:10183800F21206301205FCDFF8D2AF221217C712D7
:1018480017BF1217BF7574017575017576001125DC
:101858007C05AD5C12060BC3ED955C70F5C3E55CC9
:0E1868009401400AC3E55C94FF4037021887E4
:101876001217811216DA1217C7C2AF75EF161217B2
:10188600BFDCD10576C3E5769403500280C21217F9
:10189600BF0575E5741490009F93F808C3E5759825
:1018A600500280A91217BF1217BF0574C3E57494BE
:1018B6000C50028095120FA41216DAC2AF75EF16FD
:0318C6001217BF37
:0319FD000210FDD8
:101A00000E0915090904FF03FF0A03010155AA0184
:101A1000FFFFFFFFFF03FFFFFF25D0285004FF0259
:091A2000007AFF0101000300FF40
:101A400023475F556C74726132304123202020207F
:101A500023424C48454C492346333930232020202B
:101A60002020202020202020202020202020202076
:101C0000C2AFC2D353D9BF7581C043B20343FF8073
:101C1000752438752503B1DC7529A5752AF175E29F
:101C20004043F12053A4DF75D4FFD2857DFA7803B9
:101C300079E67C10752200752300901DE97B0675FE
:101C400024987525013085028145208508D8FBD967
:101C5000F9DCF781B7308508D8FBD9F9DCF781B713
:101C6000B19CE493A3C39A6004DDC381B7DBDBB10D
:101C70008E6002812E7B08E493FAA3B16FDBF87AC1
:101C800030B16F752200752300B18EEAFCEBFDC305
:101C9000ED94FE400EB18E8A278B28ED30E0048A49
:101CA000828B83B18E7AC270D8C3ED94FE601950D6
:101CB000CEBD002BEC600F7520007521FF7529004B
:101CC000752A000200008100A827A9280809D80465
:101CD000D90281DCB192EA89AAF281CE0D81A3C337
:101CE000ED94035053EDA2E092007AC5C3E58294CF
:101CF00000E583941C508A200010438F02438F011B
:101D00008529B7852AB7F0300029A827A92808090E
:101D1000438F01538FFDD804D902A133C3E58394C7
:101D20001C4003A3A11689AAE28529B7852AB7F02A
:101D3000A3A116538FFC817F7AC1BD030CE493A34A
:101D4000FAB153DCF8B14B817F8181AA22AB23B178
:101D50006FEBFAEA6222752608C3E52313F523E543
:101D60002213F52250066323A0632201D526EAB18F
:101D7000DCB1DC75260AEAF4200102D285300102CA
:101D8000C285B1DCC3134002C201D526EB22B19259
:101D9000EAFB208502A192308502A197752608AE44
:101DA00024AF25C3EF13FFEE13FEB1E0B1DCC3EAAD
:101DB000133085024480FA30E703632201C3E52330
:101DC00013F523E52213F52250066323A0632201B5
:101DD000D526D9E52265236523F52222AE24AF2539
:101DE0000E0FDEFEDFFCD20122424C48656C6934E6
:071DF000373164F390060196
:00000001FF
